:100000008A110A120528000009000730990083169A
:100010000510851005118312BC30A0000230A1002C
:10002000DC202F20AC012C080A3C031C2B28AD013E
:100030002D083B3C031C2528E830A0000330A1001C
:10004000DC200130AD07031C18281F308305013068
:10005000AC07031C13281F3083050C282E28051419
:100060002030A0000330A100DC20662095207920FC
:100070009520892095206B2095207F2095205C205D
:10008000A320812095207420A32074209520812016
:1000900095207D2095207020952061209520852039
:1000A0009030A0000130A100DC2005102C30A00011
:1000B0000130A100DC200800B920B920CA20B920F5
:1000C0000800B920CA20CA20B9200800B920CA20D7
:1000D000B920B9200800B920CA20CA20CA200800C7
:1000E000B920B920B9200800CA20B920CA20B920F7
:1000F0000800B920B920CA200800B9200800CA2089
:100100000800B920CA20B9200800CA20CA20CA2085
:100110000800B920B920B920B920B920080005117C
:100120004630A000A101DC20080005114630A000E7
:10013000A101DC204630A000A101DC204630A00057
:10014000A101DC20080005114630A000A101DC203F
:100150004630A000A101DC204630A000A101DC2037
:100160004630A000A101DC204630A000A101DC2027
:1001700008000515053084000230AA004B30A000AD
:100180000230A1003C30A2000030A300172105116D
:100190008F2008000515053084000230AA004B307E
:1001A000A0000230A100EE30A2000030A300172111
:1001B00005118F200800DB28A0080319E728EE208E
:1001C000A00300000000000000000000DC28A108DF
:1001D00003190800EE20A103A003DC280C30A500C1
:1001E000A50BF028000000001230A200A20BFD2891
:1001F000FF20FF20000000000800FF20F6280D303F
:10020000A400A40B0129000008001030A80200017E
:10021000031C013EA902031C08000E290A30A80293
:100220000001031C013EA902031C08000E292A0834
:1002300080042008A8002108A90005210130A2029D
:10024000031CA3032A0980052008A8002108A9008F
:100250000521A208031D1729A308031D172908005B
:02400E00C431BB
:00000001FF
